:100000000200C302EFFD120910000002EFFA000027
:1000100000000002EFF7000000000002EFF4000013
:1000200000000002EFF1000000000002EFEE00000F
:1000300000000002EFEB000000000002EFE800000B
:1000400000000002EFE5000000000002EFE2000007
:1000500000000002EFDF000000000002EFDC000003
:1000600000000002EFD9000000000002EFD60000FF
:1000700000000002EFD3000000000002EFD02020BB
:10008000434F505952494748542028432920313979
:1000900039312D31393938205041554C204E455792
:1000A0004C414E442C20502E452E20202020414CE7
:1000B0004C205249474854532052455345525645C7
:1000C000442020C2AF75D00078E0E6FBF4F60000D3
:1000D00000E6F46B70067581E00200DF7581601246
:1000E00013C4121026121422121433D2D750031242
:1000F000142C12144E121454FF24A540EBEF24BF0D
:1001000050E623C2E0FF74EDC0E07400C0E0EF9061
:10011000011D93FEEF0493C0E0EEC0E02200E8056D
:1001200076065E06F100E8097308B5085A00E80A89
:100130001500E80A3D0A74054400E80AB400E80B1B
:10014000F60AFB00E800E80C3000E80C6A00E8055D
:100150006590EF17121639221215D1AB83AC82903D
:10016000EF01EBF0A3ECF00208CA3151A3A30201A6
:10017000743151A3E0A320E70C2582F582E4358396
:10018000F58302018F2582F58274FF3583F5838024
:10019000C73151E0C4035407FDA3E0F582E5835461
:1001A000F84DF58380B23151A312163980AA31512E
:1001B00090EF17121639A3809F3151A3A380993174
:1001C00051A3A3A3809290EF09E060A580EB90EF8C
:1001D00009E0709D80E390EF0AE033409480DA906C
:1001E000EF0AE033508B80D13151A3E01201FE5071
:1001F000CE216A3151A3E01201FE40C3216AFF54AF
:100200000704FBEF54F820E7087A03C313DAFC2451
:1002100020F8B8D00790EF0AE0020233B8E0079068
:10022000EF09E0020233B8F00790EF15E002023365
:100230001213AC13DBFD223151A3E0F8E664016038
:1002400002216A21BF3151E0540704FAA3E0FB9078
:10025000EF0AE054186400700A90EF0AA3DAFDE098
:1002600002026B640014F808DAFDE66401700221F2
:10027000B9217190EF09E0FF90EF13121639E58272
:100280002FF582E43583F58321583151E0B4B4036E
:100290000202A9B4B5030202B9B4B6030202CBB498
:1002A000B7030202EB02030C2290EF09E0FB31518D
:1002B000A3E06B6002216A21BF90EF09E0FB31519E
:1002C000A3E0F8E66B6002216A21BF3151A3E0FB95
:1002D00090EF0AE05418B4000790EF0BE00202E23E
:1002E000F8E6F8E66B6002216A21BF3151A3E0FB1A
:1002F00090EF0AE05418B4000790EF0CE0020303FB
:1003000004F8E6F8E66B6002216A21BF3151E0543F
:100310000704FAA3E0FB90EF0AE05418B4000A9037
:10032000EF0AA3DAFDE002032FF81808DAFDE66B06
:10033000700221BF216A90EF16E0F8E6F58318E617
:10034000F582215801AE019101A601AE01AE01B9BD
:1003500001AE01AE01AE01AE01AE01AE01AE01AE25
:1003600001AE01AE01E8019101A601AE01AE01B9F5
:1003700001AE01AE01AE01AE01AE01AE01AE01AE05
:1003800001AE01AE01E80191033601AE01B901B938
:1003900001AE01AE01AE01AE01AE01AE01AE01AEE5
:1003A00001AE01AE01F30191033601AE01B901B90D
:1003B00001AE01AE01AE01AE01AE01AE01AE01AEC5
:1003C00001AE01AE01D6019101B901BF01B901B978
:1003D00001AE01AE01AE01AE01AE01AE01AE01AEA5
:1003E00001AE01AE01DF019101B901BF01B901B94F
:1003F00001AE01AE01AE01AE01AE01AE01AE01AE85
:1004000001AE01AE01C6019101B901BF01B901B947
:1004100001AE01AE01AE01AE01AE01AE01AE01AE64
:1004200001AE01AE01CE019101B9027301B901BF64
:1004300001B901B901B901B901B901B901B901B9EC
:1004400001B901B90171019101B901AE01AE01BF5C
:1004500001B901B901B901B901B901B901B901B9CC
:1004600001B901B901BF019101B901AE01B901B9E9
:1004700001AE01AE01AE01AE01AE01AE01AE01AE04
:1004800001AE01AE01B9019101B901AE01AE01AEFB
:1004900001B901B901B901B901B901B901B901B98C
:1004A00001B901B901B9019101B901AE028A028A0B
:1004B000028A028A028A028A028A028A028A028ADC
:1004C000028A028A01B9019101B901AE01AE01B9F6
:1004D00001AE01AE01AE01AE01AE01AE01AE01AEA4
:1004E00001AE01AE01B9019101B901AE01AE023711
:1004F00001AE01AE024502450245024502450245F4
:100500000245024501AE019101AE01AE01AE01B955
:1005100001AE01AE01AE01AE01AE01AE01AE01AE63
:1005200001AE01AE01AE019101AE01AE01AE01B965
:1005300001AE01AE01AE01AE01AE01AE01AE01AE43
:1005400001AE01AE3151E020E707239003440205DC
:1005500057C2E723900444C0E093A3F5F0D0E093A2
:10056000C0E0C0F0223151E0B4120221BF541FB4E8
:10057000110221B980CE12144EB44609120594120C
:100580001433D2D722B454091205F2121433D2D73D
:10059000220213FC12163412152112143390EF00AC
:1005A000E0640160030213FC90EF01121639E58349
:1005B000702374691213EEE5821215EF743A121368
:1005C000EE121634A8821213AC1215EF1214401258
:1005D000147A50D42274781213EE1215E4743A127D
:1005E00013EE121634E01215EF12144012147A5062
:1005F000E42212163412152112143390EF00E06435
:100600000260030213FC90EF01121639E583702794
:1006100074691213EEE5821215EF743A1213EE129A
:100620001634A88290EF04E01213981215EF1214FA
:100630004012147A50D02274781213EE1215E4741A
:100640003A1213EE12163490EF04E090EF011216F6
:1006500039F01215EF12144012147A50DA221214E3
:100660004EB4580912067C121433D2D722B4500962
:100670001206B6121433D2D7220213FC1216341209
:10068000152112143390EF00E0640260030213FCA2
:10069000A31216397C007D00E02CFC50010DA31242
:1006A0000F9050F49016F012148DED1215EFEC121D
:1006B00015EF12143322121634121521121433902E
:1006C000EF00E0640260030213FCA31216397C0001
:1006D0007D00E4932CFC50010DA3120F9050F39079
:1006E00016F012148DED1215EFEC1215EF121433F3
:1006F0002212144EB44909120727121433D2D722FA
:10070000B4580912077B121433D2D722B4500912FD
:1007100007BF121433D2D722B446091208031214A9
:100720003322D2D70213FC121634121521121433BD
:1007300090EF00E064026008E0640160030213FCD3
:10074000E490EF01F0A3A3E06006E4F0A374FFF0EF
:1007500090EF00E0FFA3121639E58254F0F582EF26
:10076000B40104120E7522B4020E120E7512147A20
:100770004005120F9050F3220213FC12163412158A
:100780002112143390EF00E064026008E06401601D
:10079000030213FC90EF00E0FFA3121639E5825428
:1007A000F0F582EFB40104120EB922B4020E120E5B
:1007B000B912147A4005120F9050F3220213FC1262
:1007C000163412152112143390EF00E06402600B0E
:1007D000E0640160060213FC90EF00E0FFA3121634
:1007E00039E58254F0F582EFB40104120EFD22B413
:1007F000020E120EFD12147A4005120F9050F322D1
:100800000213FC12163412152112143390EF00E07B
:100810006402600BE0640160060213FC90EF00E4E8
:1008200090EF01F0A3A3E06006E4F0A374FFF09062
:10083000EF00E0FFA3121639E58254F0F582EFB421
:100840000104120F4322B4020E120F4312147A4015
:1008500005120F9050F3220213FC90184012086307
:10086000D2D7227F00E4937001221213EEA3640A10
:1008700070F30FEF641470EDC082C0839008911282
:10088000148DD083D0821213E412143312143380E7
:10089000D40D0A2D2D20507265737320416E79207E
:1008A0004B657920466F72204E65787420506167E1
:1008B00065202D2D001215D11215A3600890EF1799
:1008C000EBF0A3ECF04006121521120FBF90EF0BD6
:1008D000E0A3F5F078017F06E0A3F608DFFAE0F682
:1008E000E5F0F890EF15E0F5F090EF16E0F5819067
:1008F000EF18E0C0E090EF17E0C0E090EF09E0C033
:10090000E0A3E0C0E090EF13121639D0D0D0E0227F
:10091000C082C08390EF09F0A3E5D0F075D00090BD
:10092000EF15E5F0F090EF13D0E0F0A3D0E0F090F9
:10093000EF17D0E0F0A3D0E0F090EF16E581F09053
:10094000EF0BE8F0A3E9F0A378027906E6F0A3083C
:10095000D9FA90EF171216397A0312166FDAFBE5FF
:1009600083AC8290EF17F0A3ECF0121026120D9DCD
:100970000200ED121634790090EF26121567600917
:10098000ECF0A3094003B910F2121433B90003D2FA
:10099000D7227B007C0190EF26EB4CB40003D2D72A
:1009A0002212147A5003D2D722E0F8A3AD83AE828C
:1009B0008B838C82E0A3AB83AC826870D9C082C089
:1009C00083E914FF8D838E82E0A3FAAD83AE828B20
:1009D000838C82E0A3AB83AC826A702FDFE6EB6D81
:1009E0007007EC6E7003020A0BD083D08212166F70
:1009F00074781213EEE5831215EFE5821215EFA35A
:100A0000743A1213EE121433020A0FD083D082AB61
:100A100083AC82808112163412152112143390EFA8
:100A200000E0640360030213FC90EF06E090EF0126
:100A3000121639F0A3120F9050F9D2D722121433A4
:100A400090173112148D90EF16E024F8FBF87A110C
:100A5000E81215EF12163408DAF690173712148DD3
:100A6000EBF87A11E61215EF12163408DAF61214C2
:100A700033D2D72212163412152112143390EF00FC
:100A8000E0640360030213FC90EF05121639AC8397
:100A9000AD8290EF01121639E0A3AA83AB828C835A
:100AA0008D82F0A3AC83AD828A838B82120F90502B
:100AB000E7D2D72212163412152112143390EF0008
:100AC000E0640160030213FC90EF01121639AF835A
:100AD000E58364A8FDAE82E5826458FC2D2E2FFBD1
:100AE000640FFA90EFCAEFF0A3EEF0A3EDF0A3ECE1
:100AF000F0A3EBF0A3EAF0A3D2D72212144EB4492C
:100B000009120B65121433D2D722B45809120B25DF
:100B1000121433D2D722B44609120BA9121433D2BD
:100B2000D7220213FC12163412152190EF00E0A315
:100B3000640160030213FC12163912143374781224
:100B400013EE1215E4743A1213EE121631E0121578
:100B5000EF1216341215A36002ECF020D703A38025
:100B6000D91214332212163412152190EF00E0A38B
:100B7000A3640160030213FCE0F81214331216316F
:100B800074691213EEE81215EF743A1213EE12168E
:100B900031E61215EF1216341215A36002ECF6209E
:100BA000D7030880D512143322121634121521905F
:100BB000EF00E0A3A3640160030213FCE0F8121449
:100BC0003312163474661213EE74721213EEE812B6
:100BD00015EF743A1213EE1216311213AC1215EF10
:100BE0001216341215A36004EC12139820D70308D0
:100BF00080CC12143322121634121567121433905B
:100C0000EF01EBF0A3ECF012107330D7030213FCEA
:100C100070F512166FAD83AC8290171812148DED1B
:100C20001215EFEC1215EF121433121433D2D7222F
:100C300012163412156712143390EF01EBF0A3EC87
:100C4000F01210D930D7030213FC70F512166FADF5
:100C500083AC8290171812148DED1215EFEC12155B
:100C6000EF121433121433D2D72212144EB40D06DD
:100C7000120D9DC2D722B441171214339017C81217
:100C8000148D90EF091211D2500C121433D2D722C6
:100C9000B457171214339017D012148D90EF0A1214
:100CA00011D2500C121433D2D722B44B3212143357
:100CB0009017D812148D90EF0AE0541823C412151F
:100CC000EF1216341215A3600BEC5403C403FCE0BE
:100CD00054E74CF0121433502E121433D2D722B4EE
:100CE000524A90EF0AE054186400700990EF0B121A
:100CF0001218020CFF90EF0AE05418F81212F85084
:100D000031121433D2D72290EF0AE05418640070E5
:100D10000990EF0B121221020D2490EF0AE05418F3
:100D2000F8121301500C121433D2D722B444171204
:100D3000143390182012148D90EF131211E4500CFC
:100D4000121433D2D722B442171214339018281237
:100D5000148D90EF151211D2500C121433D2D722E9
:100D6000B4531712143390183012148D90EF1612DA
:100D700011D2500C121433D2D722B450171214339C
:100D800090183812148D90EF171211E450091214B4
:100D900033D2D7220213FC121433D2D722740D128D
:100DA00013EE90EF09E01215EF121634A3E0C0E045
:100DB00012160C121634D0E01215EF121634E0544D
:100DC0001823C41215EF121634E0A35418B40028E7
:100DD0007A08E01215EF121634A3DAF612163490E0
:100DE000EF0BE0F8E61215EF121631A3E0F8E61269
:100DF00015EF121634020E19F8FF7A08E61215EFF5
:100E000012163408DAF67A02121634EFF8E6F9E729
:100E10001215EF1216340FDAEF90EF13E01215EF00
:100E2000A3E01215EF12163190EF13121639E012EB
:100E300015EF12163490EF15E01215EF121634A3C9
:100E4000E01215EF121634A3E01215EFA3E012150D
:100E5000EF12163490EF171216397A03121634E097
:100E60001215EFA3DAF612143390177812148D745A
:100E70000D1213EE22C082E582F812163174691247
:100E800013EEE81215EF743A1213EE1216347B10BB
:100E9000E6081215EF121634EB5403B401031216D0
:100EA00034DBEDD082E582F81216347B10E608A31D
:100EB00012161FDBF812143322C082C0837478121A
:100EC00013EEE5831215EFE5821215EF743A121353
:100ED000EE1216347B10E0A31215EF121634EB5409
:100EE00003B40103121634DBEDD083D08212163422
:100EF0007B10E0A312161FDBF912143322C082C04C
:100F00008374701213EEE5831215EFE5821215EF6C
:100F1000743A1213EE1216347B10E493A31215EFF9
:100F2000121634EB5403B40103121634DBECD083F5
:100F3000D0821216347B10E493A312161FDBF81232
:100F4000143322C082E582F812163474661213EE4E
:100F500074721213EEE81215EF743A1213EE1216B1
:100F6000347B101213AC081215EF121634EB540335
:100F7000B40103121634DBEBD082E582F81216348A
:100F80007B101213AC08A312161FDBF612143322C7
:100F9000FEC082C08390EF03E0FFA881E6C2D79F26
:100FA00020D714700DA318E0FFE6C2D79F20D70703
:100FB0006005D2D7020FB9C2D7D083D082EE22907B
:100FC000EF01121639E5837007E5827003020FE620
:100FD000AC83AD8212100E90EF1912101790EF0132
:100FE00012163912106790EF03121639E583700755
:100FF000E582700302100DAC83AD8212100E90EFEB
:101000001E12101790EF0312163912106722E0F922
:10101000A3E0FAA3E0FB22ECF0A3EDF0A3E9F0A338
:10102000EAF0A3EBF02290EF19121639E58370076E
:10103000E5827003021046C082C08390EF1B110E40
:10104000D083D082111D90EF1E121639E5837007F0
:10105000E5827003021066C082C08390EF20110EFB
:10106000D083D082111D227412F0A37409F0A374EE
:1010700010F0221213E4B43AFA7B001211B0FC70A3
:10108000207A041211B0DAFB7D207E00DEFEDDFA4C
:101090001213D630D7051213E480ED121433E4C3D3
:1010A000221211B0FD1211B090EF011216392582F3
:1010B000F582ED3583F5831211B01211B0F0A3DC87
:1010C000F91211B0EB600974781213EE7401D32297
:1010D000742E1213EE7401C3221213E4B43AFA7B95
:1010E000001211B0FC70207A041211B0DAFB7D20DE
:1010F0007E00DEFEDDFA1213D630D7051213E4802F
:10110000ED121433E4C3221211B0FD1211B090EFAE
:10111000011216392582F582ED3583F5831211B05F
:101120001211B0F5F0E065F06003121148A3DCF095
:101130001211B0EB600974781213EE7401D32274AB
:101140002E1213EE7401C322C082C0839011861246
:10115000148DD083D082C082C083E5831215EFE561
:10116000821215EF90119A12148DD083D082C08212
:10117000C083E01215EF9011A312148DE5F0121543
:10118000EFD083D082220D0A4572726F7220617493
:10119000206164647265737320002C20466F756E45
:1011A000643D002C2045787065637465643D2000C3
:1011B0001213E412146A1215ACC454F0F5F01213B1
:1011C000E412146A1215AC540F45F0F5F02BFBE550
:1011D000F022E01215EF1216341215A36002ECF0A3
:1011E00012143322C082C083E01215EFA3E012155F
:1011F000EF1216341215A3D083D0826005EBF0A352
:10120000ECF012143322E61215EF1216341215A365
:101210006002ECF61214332212144E121433B4305E
:1012200017C083C0829017E012148DD082D0833112
:10123000D2A3500812143322A3B43117C083C08242
:101240009017E812148DD082D08331D2A3500812A7
:10125000143322A3B43217C083C0829017F0121443
:101260008DD082D08331D2A3500812143322A3B47C
:101270003317C083C0829017F812148DD082D083A8
:1012800031D2A3500812143322A3B43417C083C040
:101290008290180012148DD082D08331D2A35008CE
:1012A00012143322A3B43517C083C08290180812D9
:1012B000148DD082D08331D2A3500812143322A3CC
:1012C000B43617C083C08290181012148DD082D00B
:1012D0008331D2A3500812143322A3B43716C0832B
:1012E000C08290181812148DD082D08331D250074A
:1012F000121433220213FC2212144E121433B4308F
:101300000F9017E012148D51060850081214332262
:1013100008B4310F9017E812148D510608500812C6
:1013200014332208B4320F9017F012148D510608AE
:1013300050081214332208B4330F9017F812148D8A
:1013400051060850081214332208B4340F901800C4
:1013500012148D51060850081214332208B4350FA8
:1013600090180812148D51060850081214332208E0
:10137000B4360F90181012148D510608500812142C
:10138000332208B4370E90181812148D51065007E6
:10139000121433220213FC22C0E090EF2374F5F004
:1013A000A3E8F0A37422F0D0E002EF23C082C08350
:1013B00090EF2374E5F0A3E8F0A37422F0D083D07B
:1013C0008202EF2375985043878075C83475CBFF30
:1013D00075CAEED29922C320980122D322C3209944
:1013E0000122D3223098FDC298E599547F2230998A
:1013F000FDC299C0E04480F599D0E02278E0E6FB98
:10140000F4F6000000E6F46B70067581E002141338
:1014100075816090170412148D1214331214330264
:1014200000E890167D12148D121497229016FD126A
:10143000148D22C0E0740D71EE740A71EED0E022BA
:10144000C0E0740D71EED0E02271E471EE2291499A
:101450001214542212146A12145E12146422B47FFD
:1014600002740822B40A02740D22FF24854009EF99
:10147000249F5004EF24E022EF2271D64001227114
:10148000E4B41B02D322B42E02D322C322E493700D
:10149000012271EEA380F69000007C007D00E493B1
:1014A0002CFC50010DA3E583B41CF3E582B4DBEE04
:1014B0009016F0918DED1215EFEC1215EF9133228D
:1014C00090EFCA121639E5824583700122E58255F4
:1014D00083F470012290EFCA7A047B00E0A32BFB17
:1014E000DAFAE0A36B600122EB650FFAE06A6001B3
:1014F0002290EFCAE0FBA3E0FAA3E064A86B6001CE
:1015000022A3E064586A6001227AFF7BFF917A503F
:101510000122DBF9DAF590EFCA121639C082C083D6
:10152000221215D17D0090EF011215676033EBF0A8
:10153000A3ECF0A30D20D7291215676024EBF0A3CC
:10154000ECF0A30D20D71A1215676015EBF0A3EC91
:10155000F0A30D20D70B1215676006EBF0A3ECF09B
:101560000D90EF00EDF022914EB4200280F97B0047
:101570007C00B40D03D3E4221215ACC0E030D704D4
:101580007B007C007A04C3EC33FCEB33FBDAF7D04E
:10159000E04CFC914EB420047401C322B40DD97404
:1015A00001D322914EB420C6E4C2D722FF24D0EF4B
:1015B00030D71824C6EF20D70394302224BFEF3051
:1015C000D70924B9EF20D7039437227400D361FCE4
:1015D00022C082C08390EF00E47A09F0A3DAFCD045
:1015E00083D08222E5831215EFE5821215EF22C027
:1015F000E0C41215FBD0E01215FB22540F24F62094
:10160000D705243A021609244171EE227F0833FEE1
:1016100040057430021619743171EEEEDFF02224A9
:10162000E030D705242030E702742E71EE22121626
:1016300034121634742071EE22C0E0C0F0E0F5F0F0
:10164000A3E0F582E5F0F583D0F0D0E022C083C0BE
:1016500082C0E0A3E004F0700612166FE004F0D040
:10166000E0D082D08322C083C082D083D08222C0C7
:10167000E01582E582B4FF021583D0E022FF110D50
:101680000A0D0A4D6F6E353120566572203938309B
:101690003131392D332E303020666F722054415055
:1016A00052205455432D35320D0A436F70797269BB
:1016B000676874202863292031393931202D2D2085
:1016C00031393938205061756C204E65776C616E08
:1016D000642C20502E452E2020416C6C20526967CE
:1016E0006874732052657365727665642E0D0A0006
:1016F000436865636B73756D3A203078006D3531E2
:101700002D3E200007202020202A2A2A2045525240
:101710004F522120000D0A005258204F4B2C2044DC
:1017200041544120454E44494E4720415420307891
:10173000004144523A20000D0A20202020202D2D67
:101740002D2D2D2D2D2D2D2D2D2D2D2D2D2D2D2DC9
:101750002D2D2D2D2D205350202D2D2D2D2D2D2D8A
:101760002D2D2D2D2D2D2D2D2D2D2D2D2D2D2D2DA9
:101770000D0A4441543A2000204120434146424250
:101780004F46502050532052422052302052312098
:1017900052322052332052342052352052362052B9
:1017A0003720405230204052312044505452204083
:1017B0004450202042205350205043545220405047
:1017C00043202B31202B320020204143433A20007C
:1017D00020205053573A200020202052423A200027
:1017E00020202052303A200020202052313A200080
:1017F00020202052323A200020202052333A20006C
:1018000020202052343A200020202052353A200057
:1018100020202052363A200020202052373A200043
:1018200020445054523A200020202020423A2000E8
:1018300020202053503A200020504354523A200098
:101840000D0A0D0A0D0A4D353120434F4D4D414EC5
:10185000445320414E442048454C502046494C4575
:101860000D0A0D0A446973706C617920504D202077
:101870002020202020202044502073746172742086
:10188000656E640D0A446973706C61792049444D3A
:10189000202020202020202044492073746172746D
:1018A00020656E640D0A446973706C617920584438
:1018B0004D20202020202020204458207374617265
:1018C0007420656E640D0A446973706C61792053ED
:1018D000465220202020202020204446207374617E
:1018E000727420656E640D0A537562737469747541
:1018F000652049444D202020202020534920616448
:101900006472202028737061636520666F72206E98
:101910006578742C20435220746F20656E64290D05
:101920000A5375627374697475652058444D20209C
:1019300020202020535820616464720D0A53756280
:10194000737469747565205346522020202020202E
:10195000534620616464720D0A6558616D696E6555
:10196000205245477320202020202020587920280D
:1019700077686572652079206973207265672C200D
:10198000737061636520666F72206E6578742C20B9
:101990002020435220746F20656E64290D0A202098
:1019A0002020202020202020202020202020202037
:1019B00020586120587720586B20587230202E2EE6
:1019C0002E205872372058642058622058732058AF
:1019D000700D0A4E65787420496E737420202020A3
:1019E0002020202020204E2028646F206F6E65204C
:1019F000696E737472756374696F6E290D0A5A6E1D
:101A000065787420496E73742020202020202020C7
:101A1000205A20286E6F20627265616B20696E20EB
:101A200063616C6C73290D0A476F20504D20202094
:101A30002020202020202020202020473C6164649A
:101A4000723E203C6270313E203C6270323E0D0A94
:101A5000525820496E74656C2020202020202020C0
:101A600020202052203C6F66667365743E0D0A4646
:101A7000696E642058444D20202020202020202002
:101A8000202046206430203C64313E203C64323EBD
:101A9000202E2E2E0D0A48656C702020202020203C
:101AA0002020202020202020204820287072696ECD
:101AB0007420746869732066696C65290D0A426C2C
:101AC00061737420544F20444D202020202020207A
:101AD000204254206164647220646174610D0A4282
:101AE0006C6173742046524F4D20444D20202020BD
:101AF0002020424620616464720D0A436865636B6E
:101B000073756D20504D2020202020202020435030
:101B100020737461727420656E640D0A4368656396
:101B20006B73756D2045444D2020202020202043DC
:101B30005820737461727420656E640D0A4C697369
:101B40007420537461636B202020202020202020EB
:101B50004C0D0A4D6F76652045444D2020202020F5
:101B60002020202020204D20737461727420656E27
:101B70006420746F0D0A4A616D2045444D20202079
:101B80002020202020202020204A2073746172749D
:101B900020656E6420646174610D0A506F77657210
:101BA000204F6E20566563746F72202020205020D5
:101BB00073746172740D0A0D0A4E756C6C20636F3C
:101BC0006D6D616E64732072657475726E207468D9
:101BD000652070726F6D707420776974686F7574AA
:101BE00020616E206572726F72206D65737361671C
:101BF000652E2020446F6E2774207573652044493C
:101C00000D0A6F7220534920746F20726561642041
:101C10006F72206D6F64696679207265676973748D
:101C20006572732E202055736520746865204558B1
:101C3000414D494E45202858792920636F6D6D61CB
:101C40006E6420696E73746561642E0D0A54797038
:101C50006963616C6C792C206D6F6E353120757302
:101C60006573205242203020666F7220776F726B4E
:101C7000696E672072656769737465727320616E3F
:101C800064207468652061637475616C2076616C92
:101C9000756573206F660D0A7468652075736572CB
:101CA000277320726567697374657273206172654A
:101CB00020617661696C61626C65207468726F7511
:101CC0006768746865206558616D696E6520636F2B
:0C1CD0006D6D616E642E0D0A0D0A00009F
:00000001FF
